:020000020000FC
:0200000003C03B
:1000060075C00FE50DBF0FE107BB002708BB00E871
:1000160000BF00270FBD0DE30EBD00E409BF05B705
:10002600006105BF552400E000936000789420919C
:100036006000203069F4C49AC09A69D0353009F05E
:100046004EC0C09801E0009360005AD0E89447C0C3
:10005600213089F45CD0323029F0C09A5CD0C09847
:100066005AD03DC0C198052D0230D4F502E0009368
:10007600600046D034C02230A9F4C19A48D032304C
:1000860009F02DC0C1980EF006C0C398539400E045
:100096000093600024C0C498C39A03E000936000F4
:1000A6002FD01DC0233059F4C29A31D0353009F013
:1000B60016C0C29804E00093600022D010C024301D
:1000C60071F425D0323029F0C29A25D0C29823D0B7
:1000D60006C0C29802E000936000689411D0A7CFD2
:1000E60005B7006205BF002708BB88950F931F93CD
:1000F6000FB7339511271FBD0FBF1F910F9118958D
:1001060000B7007F00BF00270FBD302F089500B74E
:100116000F6000BF08950F931F931FEF0FEF0A950F
:0C012600F1F71A95D9F71F910F91089579
:00000001FF
